:020000040000FA
:02000000402896
:020008000828C6
:100010008E00030E8F000B11960A250CA50C031CF5
:100020001D283A0885001F28A60A03302605240249
:10003000031C1D283A0885001F28051185110F0E85
:1000400083008E0E0E0E09000F3982077E340C34A9
:10005000B6349E34CC34DA34FA340E34FE34CE3432
:10006000EE34F8347234BC34F234E23407398207A7
:10007000803488349234AA34DA34EE34FE34FF34D7
:100080003122A00196013C3016020319AE280A3035
:100090009A00051A43289A0B4928960178301602CF
:1000A0000319AE280A309A00051E4E289A0B5428D0
:1000B0008101960123088C00002178301602031973
:1000C000AE280A309A00051A5D289A0B6328002191
:1000D000783016020319AE280A309A00051E6828E7
:1000E0009A0B6E288C0B5C2881088B120108B400D7
:1000F0001608B3008B16B730B0001B30B100B20148
:100100008D223108A0003208A10028082002031C1B
:100110008D28053C03188D28AF0A2008A8009D28CB
:100120002B08A1070318A00A2A08A0070310A00C97
:10013000A10C2008AA002108AB0020080F3C0318DE
:10014000A92820081B020318AE2820089B0018309D
:100150009E009E03031DAE2820089B002008140269
:100160000318B4283A15BB283A1DBB2814082002EE
:100170000318BB283A11200815020318C128BA1524
:10018000C828BA1DC828150820020318C828BA11A3
:10019000200813020318CE280614D528061CD528DB
:1001A000130820020318D52806101B08AE1C2008CF
:1001B00023214A082E184B082E192F082420061830
:1001C000013E86000508033903197C29412883165E
:1001D000081555308900AA30890088148818EE283F
:1001E0000811831208008900831608148312080876
:1001F00008000730C000C00BFB280800000000000A
:100200005230C000C00B022908000A30C100002192
:10021000C10B072908003230C1000021C10B0D2994
:1002200008006430C1000021C10B132908000A3006
:10023000C3001121C30B192908003230C30011215A
:10024000C30B1F290800CA01CB000A304B02031C54
:100250002C29CB00CA0A2529003403101030BC0019
:10026000CD01CE01CF01CB0DCA0DCF0DCE0DCD0DE1
:10027000BC0B3B2900344F30840045214E308400B4
:1002800045214D3084004521332903300007BD004E
:10029000BD19800030300007BD00BD1B8000003458
:1002A000CD01CE01CA014D080F39CB0067214E0E9A
:1002B00063214E0863214F0E63214F080F39CB078E
:1002C0000318CA0A08000F39CB070318CA0A03101B
:1002D0004B0DBC004A0DBD000310CB0DCA0D031021
:1002E000CB0DCA0D0310CB0DCA0D3C08CB0703186C
:1002F000CA0A3D08CA0708008B13023086000E2286
:1003000005080339033C031D802917210030F32021
:1003100023210F30B8000030B9004A081322CF0063
:10032000CF0E0930B8004B081322CF0750214B08DD
:1003300003190130880000308900E720043086006E
:100340000E220130F32023210F30B8004A08132277
:10035000CF00CF0E0930B8004B081322CF07502131
:100360004B0803190130880001308900E72008306C
:1003700086000E220230F32023210F30B8004A08F5
:100380001322CF00CF0E0930B8004B081322CF073D
:1003900050214B0803190130880002308900E72002
:1003A000103086000E220330F32023210830B800DD
:1003B0000130B9004B081322CF0050214B088800B0
:1003C00003308900E720203086000E220430F3201D
:1003D00023210730B8000030B9004B081322CF00AA
:1003E00050214B08880004308900E7204030860007
:1003F0000E220530F32023210430B8000030B9006C
:100400004B081322CF0050214B088800053089008B
:10041000E720003086000E220E2240280614172105
:10042000061017210800BC0024208600051C2B2A7A
:100430008518162ABC0A3C0838020318212A3908F4
:10044000BC003C082420013E860017210610851CB4
:10045000272A1721162A0E22051C2C2A17213C08B0
:10046000080083161330850000308600C5308100F7
:1004700083121D21BA01051185110610A801A901D9
:10048000AA01AB01A701AF019B010030F32094004A
:1004900094030130F320950095030230F32093007C
:1004A00093030330F320A3000310A30D0430F320C3
:1004B000A400A5010530F320AE0081010B118B16BD
:1004C0008B170630BC00BD013A1502308600BD0A0C
:1004D0003D083620A50017210310860DBC0B672AA6
:1004E0000630BC000730BD003A1502308600BD035F
:1004F0003D083620A50017210310860DBC0B772A76
:10050000FE308600FF30A5000614172117213A118E
:10051000061024083620A5000800B501B601B70171
:10052000300DB60D3408B6023308031C330FB50284
:100530000301031C0130B702B00D07308C00300DF1
:10054000B60DB50DB70D3408301CB02AB60233080D
:10055000031C330FB5020301031C0130B702B92A93
:10056000B60733080318330FB5070301031801302A
:10057000B707B00D8C0B9F2A310DB60DB50DB70D19
:100580003408301CCD2AB6023308031C330FB502E1
:100590000301031C0130B702D62AB607330803183B
:1005A000330FB507030103180130B707B10D07304A
:1005B0008C00310DB60DB50DB70D3408311CEA2A8B
:1005C000B6023308031C330FB5020301031C0130CC
:1005D000B702F32AB60733080318330FB507030130
:1005E00003180130B707B10D8C0BD92A320DB60DA7
:1005F000B50DB70D3408311C072BB6023308031CA8
:10060000330FB5020301031C0130B702102BB607EC
:1006100033080318330FB507030103180130B70778
:10062000B20D07308C00320DB60DB50DB70D340884
:10063000321C242BB6023308031C330FB50203010E
:10064000031C0130B7022D2BB60733080318330FF4
:10065000B507030103180130B707B20D8C0B132B3C
:100660003218382B3408B60733080318330FB50790
:02067000003454
:02400E00F23F7F
:0C42000032003200320002000500000015
:00000001FF
